:1000000012C038C018951895189518951895189518
:100010001895189518951895189518951895189578
:100020001895189518958FED8DBFC0ECE0EC4E2E0D
:10003000DD275D2EEEE7F0E0A0E6B0E088278D93A7
:100040003197E9F766248CE387BB8BEF81BB929AEB
:10005000959A939A84E690E01FD3939884E690E073
:100060001BD378948BB780648BBF85B7806385BFC3
:100070008895FBCF0F921F922F923F924F925F92E3
:100080007F92AF92BF920F931F932F933F934F9303
:100090005F936F937F938F939F93AF93BF93CF9310
:1000A000DF93EF93FF938FB78F93EFE7F0E0ABE62B
:1000B00091E01AD300916B000E3C08F004C085B7A4
:1000C000806385BF889584E690E0E6D2B09901C050
:1000D00080D1829919C0959888E290E0DDD2C49AC7
:1000E000C59A8AE090E0D8D2C5988AE090E0D4D250
:1000F000C498C59A8AE090E0CFD2C598B19901C062
:10010000E4D0B19B01C092D18F918FBFFF91EF914D
:10011000DF91CF91BF91AF919F918F917F916F911F
:100120005F914F913F912F911F910F91BF90AF9091
:100130007F905F904F903F902F901F900F90189559
:100140000895EEE7F0E0A9E6CCD20091690041E025
:10015000040FA8E60C9300916800063010F009F037
:1001600001C017C080E080936900EEE7F0E0A9E6E7
:100170007BE7A6D2959A8AEF8093640084E080930F
:1001800066005FD2829901C0FDCF84E690E084D200
:100190000895959A8AEF8093640080E080936600CA
:1001A00050D2829901C0FDCFA0E38C9182FBE6F78B
:1001B000A0E38C9182FBE6F3959888E290E06CD204
:1001C000C49AC59A8AE090E067D2C5988AE090E028
:1001D00063D2C498C59A8AE090E05ED2C59881E067
:1001E0008093610000916100003110F009F04CC073
:1001F00000916100023009F006C0009160000F3FDD
:1002000009F001C004C280E08093600080E0809328
:10021000620000916200073010F009F01BC0A0E6F8
:100220000C9142E068D24C9300916000A6E38C915F
:1002300086FB882780F9482F040FA0E60C93C59A07
:100240008AE090E029D2C598A2E68C918F5F8C93CA
:1002500008F4DFCF0091680040E14DD2A3E64C9353
:100260000091630040916100040FA3E60C93A3E6A4
:10027000EC91FF27A0E691E07BE725D2A1E68C91E7
:100280008F5F8C9308F4AECFEEE7F0E0A8E67BE753
:1002900017D284E690E000D2959A8AEF80936400AA
:1002A00081E080936600CDD1829901C0FDCFE1E06D
:1002B000F0E0E3D186E9809364000091680041E0BA
:1002C000041BA6E60C93BDD1089581E080936100E4
:1002D00000916100003110F009F03FC00091610011
:1002E000023009F006C0009160000F3F09F001C024
:1002F0008EC180E08093600080E080936200009176
:100300006200073010F009F01BC0A0E60C9142E03B
:10031000F2D14C9300916000A6E38C9186FB882774
:1003200080F9482F040FA0E60C93C59A8AE090E06C
:10033000B3D1C598A2E68C918F5F8C9308F4DFCF80
:10034000A1E6EC91FF27A0E691E07BE7BCD1A1E616
:100350008C918F5F8C9308F4BBCF84E690E09CD1A6
:10036000959A8AEF8093640081E08093660069D15A
:10037000829901C0FDCF089580E08093610080E004
:1003800080936700009167000D3710F009F00DC0F1
:10039000A7E6EC91FF27A1E691E07BE794D1A7E6E1
:1003A0008C918F5F8C9308F4EDCF80E0809369008F
:1003B000EEE7F0E0A9E67BE783D1959A8AEF809398
:1003C000640082E0809366003CD1829901C0FDCF39
:1003D000089580E08093610081E18093670000913F
:1003E00067000D3710F009F00DC0A7E6EC91FF276C
:1003F000A1E691E07BE767D1A7E68C918F5F8C93B4
:1004000008F4EDCF80E080936900EEE7F0E0A9E624
:100410007BE756D1959A8AEF8093640082E08093BF
:1004200066000FD1829901C0FDCF089580E08093CE
:100430006A0081E08093610000916100003110F05A
:1004400009F0BBC080E08093600080E08093620090
:1004500000916200073010F009F018C0A0E60C917E
:1004600042E049D14C9300916000A6E38C9186FB59
:10047000882780F9482F040FA0E60C93C59AC598E9
:10048000A2E68C918F5F8C9308F4E2CFA1E6EC9109
:10049000FF27A5E691E028D140916500009160001A
:1004A000041709F401C005C0AAE68C918F5F8C93F4
:1004B0007EC00091610040E1040FA3E60C93A3E627
:1004C000EC91FF27A5E691E00FD1409165000091E6
:1004D0006000041709F401C001C069C00091610007
:1004E00040E2040FA3E60C93A3E6EC91FF27A5E6F8
:1004F00091E0FAD04091650000916000041709F482
:1005000001C001C054C00091610040E3040FA3E6A4
:100510000C93A3E6EC91FF27A5E691E0E5D040918E
:10052000650000916000041709F401C001C03FC0DC
:100530000091610040E4040FA3E60C93A3E6EC9164
:10054000FF27A5E691E0D0D04091650000916000C2
:10055000041709F401C001C02AC00091610040E500
:10056000040FA3E60C93A3E6EC91FF27A5E691E028
:10057000BBD04091650000916000041709F401C0F0
:1005800001C015C00091610040E6040FA3E60C9382
:10059000A3E6EC91FF27A5E691E0A6D04091650087
:1005A00000916000041709F401C031C000C0A1E649
:1005B0008C918F5F8C9308F43FCF00916A000F30CD
:1005C00010F009F001C001C0BCCD959A8AEF80936C
:1005D000640081E08093660034D0829901C0FDCF31
:1005E000E1E0F0E04AD0949AE2E0F0E046D094985E
:1005F000E1E0F0E042D080916B00815080936B008D
:10060000EFE7F0E0ABE691E07BE75DD00895959AE7
:100610008AE58093640089E08093660012D080911F
:100620006B00815080936B00EFE7F0E0ABE691E068
:100630007BE749D0829901C0FDCFE1E0F0E01DD019
:10064000089580E080936100409166000091610010
:10065000041710F009F010C0939AA4E68C91992722
:100660001BD09398A4E68C91992716D0A1E68C9183
:100670008F5F8C9308F4E8CF089588EE93E00CD058
:100680003197D9F708953197F1F70895689462F892
:100690000895E89462F80895EF93FF93EE27E82B0E
:1006A000E92B31F0EAEFF0E03197F1F70197D1F75C
:1006B000FF91EF910895E199FECFEEBB3196089539
:1006C00091E001C092E07B3751F47FB7F894F3DFFB
:1006D0008D918DBBE29AE19A9A95C9F77FBF7727F2
:1006E000089591E001C092E0E6DFE09A8DB38D932A
:1006F0009A95D1F70895FF935527F8E0469508F4A9
:0E070000500F57954795FA95D1F7FF91089540
:00000001FF
